BL51 BANKED LINKER/LOCATER V5.11                                                        02/08/2014  21:32:46  PAGE 1


BL51 BANKED LINKER/LOCATER V5.11, INVOKED BY:
D:\PROGRAM FILES\KEIL\C51\BIN\BL51.EXE IIC_Send.obj TO IIC_Send RAMSIZE (64)


MEMORY MODEL: SMALL


INPUT MODULES INCLUDED:
  IIC_Send.obj (IIC_SEND)
  D:\PROGRAM FILES\KEIL\C51\LIB\C51S.LIB (?C_STARTUP)


LINK MAP OF MODULE:  IIC_Send (IIC_SEND)


            TYPE    BASE      LENGTH    RELOCATION   SEGMENT NAME
            -----------------------------------------------------

            * * * * * * *   D A T A   M E M O R Y   * * * * * * *
            REG     0000H     0008H     ABSOLUTE     "REG BANK 0"
            DATA    0008H     0002H     UNIT         _DATA_GROUP_
            IDATA   000AH     0001H     UNIT         ?STACK

            * * * * * * *   C O D E   M E M O R Y   * * * * * * *
            CODE    0000H     0003H     ABSOLUTE     
            CODE    0003H     0034H     UNIT         ?PR?MAIN?IIC_SEND
            CODE    0037H     002BH     UNIT         ?PR?_READIIC?IIC_SEND
            CODE    0062H     0026H     UNIT         ?PR?_SENDBYTE?IIC_SEND
            CODE    0088H     0020H     UNIT         ?PR?_DELAY?IIC_SEND
            CODE    00A8H     0020H     UNIT         ?PR?_WRIIIC?IIC_SEND
            CODE    00C8H     0019H     UNIT         ?PR?READBYTE?IIC_SEND
            CODE    00E1H     000CH     UNIT         ?C_C51STARTUP
            CODE    00EDH     0007H     UNIT         ?PR?DELY24?IIC_SEND



OVERLAY MAP OF MODULE:   IIC_Send (IIC_SEND)


SEGMENT                          DATA_GROUP 
  +--> CALLED SEGMENT          START    LENGTH
----------------------------------------------
?C_C51STARTUP                  -----    -----
  +--> ?PR?MAIN?IIC_SEND

?PR?MAIN?IIC_SEND              -----    -----
  +--> ?PR?_WRIIIC?IIC_SEND
  +--> ?PR?_READIIC?IIC_SEND
  +--> ?PR?_DELAY?IIC_SEND

?PR?_WRIIIC?IIC_SEND           0008H    0002H
  +--> ?PR?_SENDBYTE?IIC_SEND

?PR?_SENDBYTE?IIC_SEND         -----    -----
  +--> ?PR?DELY24?IIC_SEND

?PR?_READIIC?IIC_SEND          0008H    0002H
  +--> ?PR?_SENDBYTE?IIC_SEND
BL51 BANKED LINKER/LOCATER V5.11                                                      02/08/2014  21:32:46  PAGE 2


  +--> ?PR?READBYTE?IIC_SEND



SYMBOL TABLE OF MODULE:  IIC_Send (IIC_SEND)

  VALUE           TYPE          NAME
  ----------------------------------

  -------         MODULE        IIC_SEND
  C:0000H         SYMBOL        _ICE_DUMMY_
  D:0090H         PUBLIC        P1
  D:00A0H         PUBLIC        P2
  C:0062H         PUBLIC        _SendByte
  D:00B0H         PUBLIC        P3
  D:00A8H         PUBLIC        IE
  C:00C8H         PUBLIC        ReadByte
  D:00B8H         PUBLIC        IP
  C:0003H         PUBLIC        main
  B:00A0H.3       PUBLIC        WP
  C:0037H         PUBLIC        _ReadIIC
  D:0098H         PUBLIC        SCON
  D:0088H         PUBLIC        TCON
  B:00A0H.4       PUBLIC        SDA
  B:00A0H.5       PUBLIC        SCL
  D:00C8H         PUBLIC        T2CON
  C:00A8H         PUBLIC        _WriIIC
  C:0088H         PUBLIC        _delay
  C:00EDH         PUBLIC        Dely24
  D:00D0H         PUBLIC        PSW
  -------         PROC          _DELAY
  D:0006H         SYMBOL        x
  -------         DO            
  D:0006H         SYMBOL        i
  D:0004H         SYMBOL        j
  -------         ENDDO         
  C:0088H         LINE#         25
  C:0088H         LINE#         26
  C:0088H         LINE#         28
  C:0093H         LINE#         29
  C:00A7H         LINE#         30
  -------         ENDPROC       _DELAY
  -------         PROC          DELY24
  -------         DO            
  D:0007H         SYMBOL        i
  -------         ENDDO         
  C:00EDH         LINE#         41
  C:00EDH         LINE#         42
  C:00EDH         LINE#         44
  C:00F3H         LINE#         45
  -------         ENDPROC       DELY24
  -------         PROC          READBYTE
  -------         DO            
  D:0006H         SYMBOL        i
  D:0007H         SYMBOL        j
  -------         ENDDO         
  C:00C8H         LINE#         56
BL51 BANKED LINKER/LOCATER V5.11                                                      02/08/2014  21:32:46  PAGE 3


  C:00C8H         LINE#         57
  C:00C8H         LINE#         59
  C:00CAH         LINE#         60
  C:00CAH         LINE#         61
  C:00CCH         LINE#         62
  C:00CEH         LINE#         63
  C:00D2H         LINE#         64
  C:00D8H         LINE#         65
  C:00DAH         LINE#         66
  C:00DEH         LINE#         67
  C:00E0H         LINE#         68
  C:00E0H         LINE#         69
  -------         ENDPROC       READBYTE
  -------         PROC          _SENDBYTE
  D:0006H         SYMBOL        SendDat
  -------         DO            
  D:0005H         SYMBOL        i
  D:0003H         SYMBOL        j
  -------         ENDDO         
  C:0062H         LINE#         80
  C:0064H         LINE#         81
  C:0064H         LINE#         83
  C:0066H         LINE#         84
  C:0066H         LINE#         85
  C:0068H         LINE#         86
  C:006CH         LINE#         87
  C:006FH         LINE#         88
  C:0071H         LINE#         89
  C:0074H         LINE#         90
  C:0076H         LINE#         91
  C:007AH         LINE#         92
  C:007EH         LINE#         93
  C:0080H         LINE#         94
  C:0083H         LINE#         95
  C:0085H         LINE#         96
  C:0087H         LINE#         97
  -------         ENDPROC       _SENDBYTE
  -------         PROC          _WRIIIC
  D:0007H         SYMBOL        Wcmd
  D:0008H         SYMBOL        add
  D:0082H         SYMBOL        dat
  C:00A8H         LINE#         108
  C:00AEH         LINE#         109
  C:00AEH         LINE#         110
  C:00B0H         LINE#         111
  C:00B2H         LINE#         112
  C:00B4H         LINE#         113
  C:00B6H         LINE#         114
  C:00B9H         LINE#         115
  C:00BEH         LINE#         116
  C:00C3H         LINE#         117
  C:00C5H         LINE#         118
  C:00C7H         LINE#         119
  -------         ENDPROC       _WRIIIC
  -------         PROC          _READIIC
  D:0007H         SYMBOL        Wcmd
  D:0008H         SYMBOL        add
BL51 BANKED LINKER/LOCATER V5.11                                                      02/08/2014  21:32:46  PAGE 4


  D:0082H         SYMBOL        Rcmd
  -------         DO            
  D:0007H         SYMBOL        i
  -------         ENDDO         
  C:0037H         LINE#         130
  C:003DH         LINE#         131
  C:003DH         LINE#         133
  C:003FH         LINE#         134
  C:0041H         LINE#         135
  C:0043H         LINE#         136
  C:0045H         LINE#         137
  C:0048H         LINE#         138
  C:004DH         LINE#         139
  C:004FH         LINE#         140
  C:0051H         LINE#         141
  C:0053H         LINE#         142
  C:0055H         LINE#         143
  C:005AH         LINE#         144
  C:005DH         LINE#         145
  C:005FH         LINE#         146
  C:0061H         LINE#         147
  C:0061H         LINE#         148
  -------         ENDPROC       _READIIC
  -------         PROC          MAIN
  -------         DO            
  D:0001H         SYMBOL        i
  D:0003H         SYMBOL        get
  -------         ENDDO         
  C:0003H         LINE#         159
  C:0003H         LINE#         160
  C:0003H         LINE#         162
  C:0005H         LINE#         163
  C:0007H         LINE#         164
  C:0017H         LINE#         166
  C:0019H         LINE#         167
  C:0019H         LINE#         168
  C:0028H         LINE#         169
  C:002AH         LINE#         170
  C:0031H         LINE#         171
  C:0035H         LINE#         172
  -------         ENDPROC       MAIN
  -------         ENDMOD        IIC_SEND

Program Size: data=11.0 xdata=0 code=244
LINK/LOCATE RUN COMPLETE.  0 WARNING(S),  0 ERROR(S)
